:020000040800F2
:10000000180B0020B9020008431E0008251D000837
:10001000411E00088D1000081D240008000000008B
:10002000000000000000000000000000D1220008D5
:100030001711000800000000B9200008692300081B
:10004000D3020008D3020008D3020008D30200083C
:10005000D3020008D3020008D3020008D30200082C
:10006000D3020008D3020008D3020008D30200081C
:10007000D3020008D3020008D3020008D30200080C
:10008000D3020008D3020008D3020008D3020008FC
:10009000D3020008D3020008D3020008D3020008EC
:1000A000D3020008D3020008D3020008D3020008DC
:1000B000D3020008D3020008D3020008D3020008CC
:1000C000D3020008D3020008D3020008D3020008BC
:1000D000D3020008D3020008D3020008D3020008AC
:1000E000D3020008D3020008D3020008D30200089C
:1000F000D3020008D3020008D3020008D30200088C
:10010000D3020008D3020008D3020008D30200087B
:10011000D3020008D3020008D3020008D30200086B
:10012000D3020008D3020008D3020008D30200085B
:10013000D3020008D3020008D3020008D30200084B
:10014000D3020008D3020008D3020008D30200083B
:10015000D3020008D3020008D3020008D30200082B
:10016000D3020008D3020008D3020008D30200081B
:10017000D3020008D3020008D302000800000000E8
:10018000D3020008D3020008D3020008D3020008FB
:10019000D3020008D3020008D3020008D3020008EB
:1001A000D3020008D3020008D3020008D3020008DB
:1001B000D3020008D3020008D3020008D3020008CB
:1001C000D3020008D302000800F002F800F04BF858
:1001D0000AA090E8000C82448344AAF10107DA45A2
:1001E00001D100F040F8AFF2090EBAE80F0013F0A9
:1001F000010F18BFFB1A43F0010318472C2400001D
:100200004C240000103A24BF78C878C1FAD85207AD
:1002100024BF30C830C144BF04680C607047000080
:100220000023002400250026103A28BF78C1FBD8FF
:10023000520728BF30C148BF0B607047642900F0E7
:100240001381002070471FB502F0D4F99DE8030028
:1002500000F00CFD00F059F900F046FA1FBD10B592
:1002600000F0ABFA10BD00F0DBFA1146FFF7EBFF30
:1002700002F05CF900F0CAFC03B4FFF7F0FF03BC26
:1002800000F06EFE0B49D1F800C04A685CF8043BF0
:100290001068184442F8040B8C4528BFA1F1DC0C0F
:1002A0008A4228BFA1F1DC02C1F800C04A6020F0F8
:1002B00000407047B40300200948804709480047C0
:1002C000FEE7FEE7FEE7FEE7FEE7FEE7FEE7FEE706
:1002D000FEE7FEE704480549054A064B7047000063
:1002E0000D240008C901000818050020180B002083
:1002F000180700201807002053EA020C00F069805C
:100300002DE9F04B4FF00006002B1FBFB3FA83F529
:1003100003FA05F424FA05F65E4012BF1643B2FA5A
:1003200082F502FA05F4C5F120051EBF22FA05FC8C
:1003300044EA0C04203556EA044C4FEA144418BF32
:10034000641C4FF000084FF00009904271EB030C61
:1003500039D3002919BFB1FA81F701FA07F6B0FACB
:1003600080F700FA07F6C7F120071EBF20FA07FC46
:1003700046EA0C062037B6FBF4FCA7EB0507103F56
:1003800007F01F0BCBF120060CFA0BFB2CFA06F63C
:1003900044BFB3460026202FA4BF5E464FF0000B9B
:1003A0005BEA060C08BF4FF0010B19EB0B09ABFB26
:1003B000027C48EB0608C01B06FB02CC0BFB03CCFF
:1003C00071EB0C01C1E70B46024641464846BDE8C9
:1003D000F08B13B54FF000004FF00001AFF3008039
:1003E000BDE81C40704700000FB4044910B503AAD3
:1003F000029800F04BF910BC5DF814FB10040020CB
:100400002DE9F0410E460446002020622046E168B6
:10041000884730B3252805D0D4E901219047206AC8
:10042000401CF2E7E168204600278847050018D005
:10043000A5F14100192802D820354FF40067324653
:10044000294620462760FFF7F9FE40B1012804D075
:10045000F61D26F007060836D8E7361DD6E72846EB
:10046000DAE7206ABDE8F0812DE9F0410646002474
:1004700010687529314616A510D0AFF3008000280A
:1004800002DA404213A507E031688A0701D512A5B8
:1004900002E0490704D511A5012401E0AFF3008073
:1004A00000210A2206F1240709E0B0FBF2FCB0FBB0
:1004B000F2F302FB1C00303078541846491C002827
:1004C000F3D123462A463046BDE8F04100F085B816
:1004D000000000002D0000002B00000020000000A4
:1004E0000B4910B5A1F17C020A4CC2E93712372141
:1004F00006E000EB104342F82130074B00FB0340BD
:100500000B1EA1F10101F4DC10BD0120E8E70000A1
:1005100054030020E119D666CD0D01004FF0000212
:1005200000B5134694469646203922BFA0E80C50E9
:10053000A0E80C50B1F12001BFF4F7AF090728BFC4
:10054000A0E80C5048BF0CC05DF804EB890028BF40
:1005500040F8042B08BF704748BF20F8022B11F069
:10056000804F18BF00F8012B704700004FF0013C8E
:1005700050F8042B51F8043B9A4215D1A2EB0C031E
:10058000934313EACC130BD150F8042B51F8043BDE
:100590009A4209D1A2EB0C03934313EACC13E7D0A0
:1005A0004FF00000704700BFD01A01BAB1FA81F1D4
:1005B00001F0180122FA01F0CB40C1F12001DBB2B9
:1005C000C0B2C01A2CFA01F3D11A914311EAC31137
:1005D000E6D170477047704770472DE9F0470D46E8
:1005E00099469246044600F124080168880604D51D
:1005F000E06921F01001216000E00120A84201DD46
:10060000471B00E00027A1697A1902EB0900081ACC
:10061000A0612078C00602D42046AFF300800026F7
:1006200008E0D4E901211AF806009047206A401C2E
:10063000761C20624E45F4DB2078C0060AD52046A1
:10064000AFF3008006E0D4E9012130209047206A12
:10065000401C2062381EA7F10107F4DC07E0D4E952
:10066000012118F805009047206A401C2062281ECE
:10067000A5F10105F3DC2046AFF3008020780006E9
:1006800002D50220BDE8F0870120FBE7074B70B5DB
:100690000D467B4400F011F80446284600F020F88F
:1006A00010B14FF0FF3070BD204670BD7B1E0000C2
:1006B00001694A1C02610878704700B58FB0CDE926
:1006C00001310021059105497944CDE90310114616
:1006D0006846FFF795FE0FB000BD0000E5FFFFFF85
:1006E000007B00F08000704710B542485421FFF7AE
:1006F00015FF41485421FFF711FF40485421FFF7EF
:100700000DFF3F493B483C4A3F4B08603D490A606A
:100710003A491960531C0365481C1065012008659F
:100720003B48344A39A1784400F0D4F920B938481C
:1007300078440A3800F073FA37482F4A35A17844D4
:1007400000F0C8F920B9344878440A3800F067FA54
:1007500032482A4A2FA1784400F0BCF920B92F482A
:1007600078440A3800F05BFA40232248DC0000217C
:10077000224600F08CF920B125487844543800F026
:100780004EFA1D4822464023002100F080F920B196
:1007900021487844543800F042FA18482246102381
:1007A000002100F074F9002806D01C487844BDE808
:1007B0001040563800F033BA10BD104870B5006DC7
:1007C00020F001040B4800F0FBF90B4800F0F8F9A9
:1007D0000A4800F0F5F909E0206D20F001052046F7
:1007E00000F0EEF9204600F040F82C46002CF3D142
:1007F00070BD0000BC030020100400206404002031
:1008000020000020240000202800002072000000AA
:10081000D41E000077000000C31E0000B31E0000BD
:10082000754600F003FAAE4605006946534620F0CF
:100830000700854618B020B5FFF74CFDBDE8204005
:100840004FF000064FF000074FF000084FF0000B8C
:1008500021F00701AC46ACE8C009ACE8C009ACE83F
:10086000C009ACE8C0098D46704770B50446051F45
:1008700000F0E0F90068002C14BF446870BD002C43
:1008800018BFAC423CBF20466468F8D301680A1820
:10089000AA4218BF456003D12A6805461144016089
:1008A00028684119A1421CBF6C6070BD6168696015
:1008B00021680844286070BD2DE9F04705460C46C4
:1008C000C86820F4201040F48000C860800602D57B
:1008D000084600F0FCFAE06841F282014FF0FF396F
:1008E0000140022903D0204600F09AFAB5E000F456
:1008F0002041B1F5004F0FD1C00306D56168E06A11
:10090000884200D80846606006E02069E0626060C6
:10091000606901F0A1FDA061A0680022EEB200288C
:100920000DDAE1688B050AD4C043A06041F4903031
:100930002260E0606068411C61600670A5E0E068CC
:100940009046226040F40050E060206968BB606916
:1009500001F088FD012704F12405A0B1A08910F45D
:10096000407F08D0E06900F0B0F9206118B1E0687C
:1009700040F4006016E0E7612561E06820F4407013
:1009800040F480600EE0E06900F09FF900282061EB
:10099000F1D0E06840F4006010F4407FE06002D1E4
:1009A00040F48070E06020696060E06825696FF065
:1009B000010AC1051FD56168E06A884200D808466F
:1009C000411B04D02246284600F034FAF0BBE06810
:1009D000010203D5E562C4E9015854E0691CE162F3
:1009E0006160E16940F48030491EC4E9021030467C
:1009F0002E70BDE8F087010202D500F480320AE0D3
:100A00006068411C61600670E0680A2E40F4803026
:100A1000E06006D00022E16A6068814203D90B469B
:100A200002E00122F7E70346A7895B1B7F0503D499
:100A3000E7699F4200DDE2B1814200D80146E562EC
:100A40000F1AC4E90158002B09DD00E005E0224639
:100A50001946284600F0EEF908B14846C9E747B103
:100A6000A069E5626560C01BA061E06840F010000D
:100A7000E060E068000208D56168A069E562491B92
:100A800008446560A0615046B3E73046B1E770B5F1
:100A9000C468A50713D0650211D4B2F5807F09D0D0
:100AA000B2F5007F06D0B2F5806F08D1012300F1C6
:100AB000240106E05D1E6FF07F46B54201D30120A0
:100AC00070BD0161C361416024F470611143C16074
:100AD000002070BD2DE9F0410C4607461646104631
:100AE00000F06EF82078611C61280AD0722802D0CC
:100AF00077283CD102E00125002405E002250424EA
:100B000002E0082448F2020511F8010B2B2806D058
:100B1000622809D011F8010C74280AD00BE045F0C6
:100B2000030544F00204EFE745F0040544F0010436
:100B3000EAE744F010043846214601F09FFC411CCE
:100B400015D00021316171604FF40071F560F161E1
:100B50007061200704D530460222002100F0E4F83D
:100B6000306D40F0010030653046BDE8F081002076
:100B7000FBE72DE9F0410D460646104C206DC107FC
:100B800004D0410804D020F00104F7E722460EE02B
:100B9000542000F09AF807000ED0206D47F00101B4
:100BA0000843542120653846FFF7B8FC3A462946E9
:100BB0003046BDE8F0418DE70020D6E7BC030020B9
:100BC0002DE9F04704464FF000094FF0FF37C568A4
:100BD000D4E90486A80707D0204600F055F930462E
:100BE00001F02EFC002802DA3846BDE8F08728051F
:100BF00002D54046FFF739FE4C212046FFF78EFC18
:100C0000206D20F0010020654846EEE710B504464F
:100C1000AFF300802046BDE81040FFF72DBB10B5B4
:100C200000F07CF9BDE8104000F072B90048704750
:100C3000B804002000487047C00400207047704787
:100C40007047704738B504460A4600206946AFF33E
:100C50000080002808BF38BD02460099204600F0F9
:100C60008DF9012038BD012000F072B9F8B5AFF35D
:100C70000080054600200C46102000BF0646A8193B
:100C8000A0420DD9324669460020AFF3008007002C
:100C900008BF00F05DF90098A04218BF0546C419CE
:100CA000FFF7C8FF05600746F01D20F00700461952
:100CB000284600F05CF9B44208BFF8BDA21B3146DB
:100CC0003868BDE8F84000F059B970B50646FFF73E
:100CD000B1FF056806F10B0020F00704B4429CBF89
:100CE000002070BD2B466A68BAB11068A04210D3CC
:100CF00004F1080188423CBF5068586007D351682E
:100D0000101941601168091B016058601460101DC2
:100D100070BD13465268002AE7D121462846FFF7E6
:100D200091FF0028DED170BD2DE9F0410446164642
:100D30000D464769007B80072ED0384601F092FBB4
:100D400050BB3EB3012E02D0022E25D104E0204636
:100D500000F02EF905441DE0384601F07DFBE16806
:100D6000002841F01001E16005DA204600F058F853
:100D70000120BDE8F081C9030BD56268E16A9142A8
:100D800000D81146A26911442269891A814200DD06
:100D900008460544002D01DA0220EAE7E16A6068AE
:100DA000E268814206D29103E06203D522F4003169
:100DB00041F01002A6690027AE4213DCE16A8142CD
:100DC00001D90B4600E0034603EB060C2369ACEBAC
:100DD000030CAC4506DD814201D98C4600E0844617
:100DE0009C4505D1A760276042F02000A5620DE078
:100DF000AD1BE669AE1B8142A66000D90846C01A49
:100E0000281A20605819606022F020000349084029
:100E1000E060002084F84870ABE70000BFCFD7FF48
:100E2000C16821F4001141F08001C160002181609E
:100E3000016070472DE9F047814614460E464FF099
:100E4000FF383248D5685769054209D03846A1694C
:100E500001F042FB002811DB2C48C0430540E5604F
:100E60002B4632464946384601F03BFBA16920F04B
:100E70000042B21A11440028A16103D02046FFF7B6
:100E8000CFFF4046BDE8F08770B504460569C06AEB
:100E90006168884200D80846E16821F42011E160C9
:100EA000C90312D5A84208D02246411B2846FFF7A5
:100EB000C1FF10B14FF0FF3070BD0020E562C4E902
:100EC0000150E06820F48030E060002070BD10B573
:100ED0000446C06820F02000E060A16AA069884252
:100EE0000DD02046FFF7D0FFE06820F4405040F0DE
:100EF0001000E060A06AA0612069E062606044F2D6
:100F00004001E0688843E06010BD0000100002006E
:100F1000002801D000F024B87047000010B5014649
:100F200002A000F066F8012010BD000053494752AE
:100F3000545245443A2052656469726563743A209C
:100F400063616E2774206F70656E3A2000000000A8
:100F500010B500F067F8BDE81040FFF7D9BF0000FA
:100F600001491820ABBEFEE72600020070470021B1
:100F70000160C0E9011070471020704703464068C7
:100F80008C46002818BF88423CBF03464068F8D30F
:100F900018681844884207D00CF1030020F00700BD
:100FA000001D411A521A0146081D0A60FFF75DBC78
:100FB00010B50146C268900703D0900607D5886A2D
:100FC0000AE000F05FF801210160881E10BD8B6906
:100FD000486818440B69C01A91F848301BB191F861
:100FE0004910401A10BD1103FCD50028FADD401E3F
:100FF00010BD70B505460C460A2000E06D1C00F0DF
:1010000039F835B128780028F8D102E0641C00F0E6
:1010100031F814B120780028F8D1BDE870400A20DA
:1010200000F028B810B5012805D0002103A0FFF773
:10103000E0FF012010BD09A1F8E700005349475225
:10104000544D454D3A204F7574206F662068656198
:1010500070206D656D6F7279000000003A20486560
:101060006170206D656D6F727920636F727275703B
:101070007465640008B569468DF800000320ABBEB6
:1010800008BD000000487047B8040020FEE770B5B6
:101090000C4691F9001005460078084440B25428E7
:1010A00017D300296FF0004607DDFFF7EBF800EBE0
:1010B000400090FBF6F0C04306E0FFF7E3F800EBDA
:1010C000400090FBF6F0401C2070287821780844FE
:1010D00040B2287070BD70B50C4691F900100546FD
:1010E0000078084440B2302813D300296FF000463E
:1010F00005DDFFF7C7F890FBF6F0C04304E0FFF70B
:10110000C1F890FBF6F0401C207028782178084444
:1011100040B2287070BD704772B6FEE72DE9F84FF7
:10112000DFF80CB2012403254FF00F0A00220BF167
:10113000040E00BF0B6804FA02F63340B34278D1C4
:101140000F7907F00307012F01D0022F1AD187680A
:101150004FEA4209D1F80CC005FA09F827EA080756
:101160000CFA09FC4CEA070CC0F808C0476891F873
:1011700004C0B743CCF3001C0CFA02FC4CEA070C89
:10118000C0F804C00E79F643B6070BD0C6684FEA24
:10119000420C8F6805FA0CF826EA080607FA0CF7E5
:1011A0003743C7600E7906F00306022E12D1D60827
:1011B0004FEA427800EB860600960F69D6F8209039
:1011C0004FEAD8660AFA06FCB74029EA0C0637430C
:1011D000009E37620F7906684FEA420C07F003075A
:1011E00005FA0CF807FA0CF726EA080637430760F9
:1011F0004E6816F4403F1CD04E4E376847F4804787
:101200003760366822F00308970706F48046009698
:10121000494E3F0F4644B146D6F80868DFF81C81B6
:101220000AFA07FC404526EA0C0603D14FF0000CF1
:1012300041E076E0DFF808C1604502D14FF0010CD3
:1012400039E0DFF800C1604502D14FF0020C32E016
:10125000DFF8F4C0604502D14FF0030C2BE0DFF85B
:10126000ECC0604502D14FF0040C24E0DFF8E0C090
:10127000604502D14FF0050C1DE0DFF8D8C0604595
:1012800002D14FF0060C16E0DFF8CCC0604502D169
:101290004FF0070C0FE0DFF8C4C0604502D14FF0FB
:1012A000080C08E0DFF8B8C0604502D14FF0090C27
:1012B00001E04FF00A0C0CFA07FC4CEA060CC9F8E6
:1012C00008C84F68DBF80060FF0226EA030600D575
:1012D0001E437746CBF80060D1F804C0DEF800600A
:1012E0005FEA8C2C26EA030600D51E43DFF840C0D7
:1012F0003E60ACF1040C4F68DCF80060BF0326EAE6
:10130000030600D51E430A4FCCF80060083FD1F811
:1013100004C03E685FEACC3C26EA030600D51E43C3
:101320003E60521C102AFFF405AFBDE8F88F0000A4
:10133000083C0140443802400030014000000240B7
:101340000004024000080240000C0240001002406D
:101350000014024000180240001C0240002002401D
:10136000002402400AB1816170470904FBE70000D4
:101370000148806870470000100000200248816822
:10138000027811448160704710000020032010B5DE
:1013900000F060F80F2000F005F800F023F80020BE
:1013A00010BD000070B50D4D04464FF47A700C4A24
:1013B00029781268B0FBF1F0B2FBF0F000F09FFC6E
:1013C00048B9102C07D200222146501E00F022F806
:1013D00000206C6070BD012070BD00001000002076
:1013E0001C0000200A4808B5016841F080510160E6
:1013F000006800F0805000900548001D016841F42D
:1014000080410160006800F48040009008BD000049
:10141000403802400E4BF0B41B680D46C3F3022364
:10142000C3F10706042E00D90426191D072901D28D
:10143000002300E0DB1E012404FA06F19C40491E53
:101440002940641E994014402143F0BC00F0E7BFDE
:101450000CED00E0064900F0070210B54FF6FF045E
:101460000868044B204040EA02201843086010BD81
:101470000CED00E00000FA051848F8B5016841F0ED
:10148000805101600068164C00F080500090206888
:1014900040F480302060FFF76BFF4FF47A7605460A
:1014A00005E000BFFFF764FF401BB0420FD8606843
:1014B000C003F7D5206840F400302060FFF758FFE4
:1014C000054606E0FFF754FF401BB04201D9032058
:1014D000F8BD60688003F5D50020F8BD40380240B3
:1014E000007000402DE9F04705000F4663D0444EE0
:1014F000306800F00F00B84209D2306820F00F00C9
:1015000038433060306800F00F00B84253D128688B
:101510003C4C810712D5400703D5206840F4E050C9
:1015200020602878000703D5206840F460402060E0
:10153000A968206820F0F000084320602878C007E0
:101540002AD0304968680839012810D00968022873
:1015500010D0890700292EDA216821F00301014308
:101560002160FFF705FF804641F288390DE00968E8
:101570008903EFE78901EDE7FFF7FAFEA0EB080129
:10158000494502D90320BDE8F0876868216801F069
:101590000C01B1EB800FEFD1306800F00F00B842C2
:1015A0000BD9306820F00F0038433060306800F00D
:1015B0000F00B84201D00120E5E72878400705D5A3
:1015C000E968206820F4E05008432060287800078C
:1015D00006D52869216821F4604141EAC0002060F5
:1015E00000F018F82168084AC1F30311515CC840A3
:1015F0000649086006480068FFF7D4FE0020C2E7ED
:10160000003C024008380240152600081C0000205B
:1016100014000020154910B51548096811F00C0296
:1016200013D01449042A0FD0082A0ED10F4C241FBE
:101630002268236802F03F025B0207D52068C0F3EE
:101640008810A0FB010106E0084610BD2168C1F327
:101650008811A1FB00010023FEF74EFE2168C1F3B3
:101660000141491C4900B0FBF1F010BD08380240AF
:101670000024F40040787D012DE9F84F04004FF07C
:1016800000076ED02078DFF868A3AAF10408C0072D
:10169000A8F104054CD0DAF800105046C1F38101DE
:1016A000012908D00068C0F3810002280AD1D8F8C7
:1016B0000000400206D52868800339D560680028FC
:1016C000DFD035E06068B0F5803F0BD010B1B0F5E9
:1016D000A02F11D0286820F480302860286820F4DA
:1016E000802002E0286840F480302860606890B173
:1016F000FFF73EFE06460AE0286840F48020286096
:10170000F0E700BFFFF734FE801B642872D828681A
:101710008003F7D50CE0FFF72BFE064605E000BF7F
:10172000FFF726FE801B6428F0D828688003F7D4D2
:101730002078800742D5DAF80010504611F00C0FDF
:1017400008D00068C0F3810002280BD1D8F800004F
:10175000400207D42868800718D5E068012800D126
:1017600014E041E1E0680028286817D040F001004B
:101770002860FFF7FDFD064605E000BFFFF7F8FD16
:10178000801B0228C2D828688007F7D520692968FD
:1017900021F0F80141EAC00028600FE020F00100CC
:1017A0002860FFF7E5FD064605E000BFFFF7E0FD16
:1017B000801B02281ED828688007F7D420780007ED
:1017C00029D58B4861696C3000298146016812D0A7
:1017D00041F001010160FFF7CBFD064605E000BFC7
:1017E000FFF7C6FD801B022804D8D9F80000800747
:1017F000F6D510E089E021F001010160FFF7B8FDA6
:10180000064604E0FFF7B4FD801B02287DD8D9F816
:1018100000008007F6D4207840076BD5DFF8D09120
:1018200009F13809D9F80000C0000BD4D9F800102C
:1018300041F08051C9F80010D9F80000012700F0EC
:10184000805000906B480168C90512D40168834636
:1018500041F480710160FFF78BFD064605E000BF93
:10186000FFF786FD801B64284FD8DBF80000C00519
:10187000F6D55F4EA068683601280AD008B1052861
:1018800011D0306820F001003060306820F0040092
:1018900002E0306840F001003060A068A0B1FFF7BE
:1018A00067FD83460CE0306840F004003060F0E7EC
:1018B000FFF75EFDA0EB0B0141F28830814266D854
:1018C00030688007F4D50EE0FFF752FD834607E04D
:1018D000FFF74EFDA0EB0B0141F28830814256D854
:1018E00030688007F4D42FB1D9F8001021F080516E
:1018F000C9F80010A069C8B3DAF80010C1F381017B
:1019000002294BD00228286800E040E020F08070D7
:10191000286003D0FFF72CFD04463BE0FFF728FDCD
:10192000064604E0FFF724FD801B02282FD8286814
:101930008001F7D4D4E90962D4E907012E4B570896
:1019400094F82C20084303EB074343EA861108432D
:1019500040EA026040F00050C8F80000286840F0FB
:1019600080702860FFF704FD044606E03EE000BFFB
:10197000FFF7FEFC001B022809D828688001F7D574
:1019800034E000BFFFF7F4FC001B022802D903205B
:10199000BDE8F88F28688001F4D427E00128D8F842
:1019A000000021D0E16900F480028A421CD1216A42
:1019B00000F03F028A4217D1626A47F6C0710140C7
:1019C000B1EB821F10D1A16A4FF0FF3200F4403317
:1019D00002EB5101B3EB014F06D194F82C1000F04B
:1019E0007060B0EB016F01D00120D1E70020CFE79C
:1019F00008380240007000400000FFFF2DE9F04170
:101A000004000AD0606A002550B12561C4F8145062
:101A100094F85D00A56248B10DE00120BDE8F081B9
:101A20006068B0F5827FF3D0E561F1E7204684F885
:101A30005C5000F05DF8022084F85D004FF4E06235
:101A40002068016821F040010160E068904201D9FE
:101A5000002101E04FF48051B0F5706F02D0904248
:101A600000D0A5622289A088237C02F4044C277D43
:101A700000F4827003F00206228B40EA0C00237F00
:101A8000304394F8206007F001073843278D02F4B3
:101A90000072104303F038031843236806F08002F5
:101AA000104307F4005630431860A069042394F8EB
:101AB000242001F4805194F8346003EA1040A7898F
:101AC00002F01002104306F008031843236807F4DD
:101AD00070621043084358602068C16921F40062B5
:101AE000C2610121256684F85D10002096E70000A0
:101AF000F0B587B0044614216846FEF70FFD1A4979
:101B0000206888422ED11948016841F48041016063
:101B1000006800F48040059014481038016841F4D2
:101B200080710160016801F480710591016841F0E4
:101B300002010160006802240527009400F0020001
:101B4000694601AA0025CDE904700326084882E809
:101B50007000FFF7E3FAA00369468DE8F10005483D
:101B6000FFF7DCFA07B0F0BD003800404038024013
:101B700000200240000402402DE9F84F044690F88E
:101B80005C0000271D460128164689460DD04FF0FF
:101B9000010B84F85CB0FFF7EBFB804694F85D0026
:101BA000BA46012804D00227A3E00220BDE8F88F3E
:101BB000B9F1000F73D0002E71D0A2680321C4F8D0
:101BC0003890A68784F85D10C4F860A0E687C4F852
:101BD00040A0A4F844A0A4F846A0B2F5004FC4F871
:101BE00050A0C4F84CA009D12068016821F0400140
:101BF00001602068016841F480410160206801684B
:101C0000490603D4016841F040010160E068B0F585
:101C1000E06F606823D908B1012E1CD1A06B216848
:101C20000088C86006E020688168890709D5A16B33
:101C30000988C160A06B801CA063E08F401EE08714
:101C400009E0FFF795FBA0EB0800A84202D3681C4F
:101C500001D045E0A5B3E08F0028E4D135E008B11C
:101C6000012E2FD1E08F21680128A06B02D90088B6
:101C7000C8600EE00078087314E0E08722E0206876
:101C80008168890714D5E18F0129A16B08D90988DA
:101C9000C160A06B801CA063E08F801EEDE727E091
:101CA00009780173A06B401CA063E08F401EE4E73D
:101CB000FFF75EFBA0EB0800A84202D3681C01D02E
:101CC0000EE06DB1E08F0028D9D14246294620466A
:101CD00000F0F4F908B120202066A06810B105E0FA
:101CE000032706E02068C16880680090206E00B17C
:101CF000012784F85DB0384684F85CA056E7401EA2
:101D0000B0F1807F10B501D3012010BD4FF0E02469
:101D100060610F21601700F082FB0020A0610721A5
:101D2000216110BDFEE7000007490968C9070AD014
:101D3000054980390968C90705D04FF060410A6834
:101D4000002AFCD008707047800E00E0F0B587B024
:101D500014216846FEF7E2FB2248016841F00201C7
:101D60000160016801F002010591016841F4807190
:101D70000160016801F480710591016841F0200162
:101D8000016000680022184E4FF4407100F02000FE
:101D900005903046FFF7E6FA144F002240213846FE
:101DA000FFF7E0FA0124694600252002CDE900048E
:101DB000CDE902453046FFF7B1F9022103956002F3
:101DC00000903046CDE901416946FFF7A7F9402070
:101DD0006946CDE90004CDE902453846FFF79EF992
:101DE00007B0F0BD30380240000402400014024049
:101DF00070B512484FF4E06400210F4E4FF4827525
:101E00001823C0E9021401617215E0E80565072492
:101E1000082580E80E00C1600161C0E90514C0E931
:101E200007150648FFF7EAFD002803D0BDE870401B
:101E3000FFF772B970BD0000003800407402002046
:101E4000FEE7FEE730B5532813D82F2911D8CC0868
:101E50000123C4EBC40401F0070104EB4405064C64
:101E60008B4000EB8500002A21680A5C02D01A43EF
:101E70000A5430BD9A43FBE70C000020F1B50F4D2A
:101E80004FF40074002221462846FFF76BFA0C4EEF
:101E9000002240213046FFF765FA0A480A23012252
:101EA0006946FFF769FE012230464021FFF75AFAE2
:101EB000012221462846FFF755FAF8BD00040240EA
:101EC000001402407402002031B5094C0022402168
:101ED0002046FFF747FA0748002301226946FFF72B
:101EE0004BFE012220464021FFF73CFA38BD00009E
:101EF00000140240740200202DE9F04753281F46C9
:101F000016460C46DDF820A005462FD82F2C2DD8DC
:101F1000532E2BD82F2F29D8B54201D9BC4203D834
:101F2000B5423BD2BC4239D2B54203D9154606462A
:101F30001C460F46A6EB0509A7EB0408C14513DCB8
:101F400029E0711B524608FB01F0010191FBF9F0F9
:101F50000830C11700EB1170A7EB2010C1B2E8B236
:101F6000FFF770FF6D1C2DB2B542EADDBDE8F087CA
:101F7000391B524609FB01F0010191FBF8F00830D2
:101F8000C11700EB1170E1B2A6EB2010C0B2FFF751
:101F900059FF641C24B2BC42EADDE7E7B54202D92E
:101FA0001546064603E0BC4201D91C460F46A6EB87
:101FB0000509A7EB0408C14513DC15E0711B524667
:101FC00008FB01F0010191FBF9F00830C11700EBAB
:101FD000117004EB2010C1B2E8B2FFF733FF6D1CA3
:101FE0002DB2B542EADDC1E7BC4219D152462146C5
:101FF0002846BDE8F047FFF725BF391B524609FBCD
:1020000001F0010191FBF8F00830C11700EB1170ED
:10201000E1B205EB2010C0B2FFF714FF641C24B23C
:10202000BC42EADDA2E710B5044601F0070040F02B
:102030004000FFF723FF44F08000BDE81040FFF7A9
:102040001DBF0000002170B50846FFF7ECFF064DEC
:1020500000244FF4FC762868005DFFF735FF641C10
:10206000A4B2B442F7D370BD0C0000200122104886
:1020700010B51102FFF776F90E4801224021FFF753
:1020800071F92120FFF7FAFEBE20FFF7F7FE1320BB
:10209000FFF7F4FE2020FFF7F1FE0920FFF7EEFE28
:1020A0000820FFF7EBFEBDE810400C20FFF7E6BE6E
:1020B000000402400014024070470000F8B51546C5
:1020C0000E4604460B464FF4C0510092002200F029
:1020D00035F840BB17484FF47A71174A0068B0FBD7
:1020E000F2F0484300906068B0F5827F08D100228A
:1020F000334680212046009500F08EF898B908E01C
:10210000009830B1401E009020688068C0430006EF
:10211000F6D5002233464FF4C0612046009500F00A
:102120000DF8002804D0206E40F020002066032027
:10213000F8BD00001C00002000366E012DE9FE4FA6
:10214000984617460E4604460C9D4FF0000A8DF83F
:1021500004A0FFF70DF9411BA8EB0105FFF708F9F3
:1021600081462C484FF4C06B01682068C1EBC10167
:102170000C30029001EB8100000D684342E05E45A7
:1021800006D12FB9029800788DF804009DF804005C
:10219000B8F1FF3F37D0FFF7EBF8A0EB0900A842FA
:1021A00003D215B1009858B32BE02068416821F0A4
:1021B000E00141606068B0F5827F0BD1A068B0F5A6
:1021C000004F02D0B0F5806F04D12068016821F083
:1021D00040010160A06AB0F5005F09D12068016884
:1021E00021F4005101602068016841F40051016050
:1021F000012184F85D10032084F85CA0BDE8FE8F07
:102200000025401E0090206880683040B842B6D15A
:102210000020F3E71C0000202DE9F8431E469146FC
:1022200088460446089DFFF7A3F8401B351AFFF7C0
:102230009FF8074625480068C0F3CB30684338E074
:10224000701C37D0FFF794F8C01BA84203D215B119
:10225000009860B32CE02068416821F0E001416003
:102260006068B0F5827F0BD1A068B0F5004F02D056
:10227000B0F5806F04D12068016821F04001016051
:10228000A06AB0F5005F09D12068016821F400510F
:1022900001602068016841F400510160012184F867
:1022A0005D10002084F85C000320BDE8F883002561
:1022B000401E00902068816838EA010004D00021A7
:1022C0004945BDD10020F0E70121F9E71C000020BD
:1022D00070470000F8B5224C1422224D0021A0685E
:1022E000401CB0FBF2F302FB13006060009105EBB1
:1022F000800115F82000CB788A784978FFF7FCFD3B
:1023000001200090A06805EB800115F82000CB7833
:102310008A784978FFF7F0FDD4E9010105EB8000E8
:1023200005EB8101096801602146FEF7B0FE606897
:102330002646B11C05EB8000801CFEF7A8FE6068F5
:10234000711C05EB8000401CFEF7C5FE6068F11CA7
:1023500005EB8000C01CFEF7BEFE6068A060F8BD03
:10236000000000202C000020FFF708B830B593B023
:1023700030216846FEF7D2F814210CA8FEF7CEF8FB
:102380002048016841F080510160006800F08050F1
:1023900011901D48016841F440410160006800252A
:1023A0000DF1200C0224009400F44040119008220A
:1023B000D823CDE9064510218CE81C0001200B94A0
:1023C000CDE903016846FFF757F908B172B6FEE799
:1023D000FFF752F808B172B6FEE74FF480524FF49F
:1023E000A0510F20CDE90F120CAA072182E831007D
:1023F0000CA8FFF777F8002801D072B6FEE713B0FB
:1024000030BD0000403802400070004002480168C2
:1024100041F470010160704788ED00E0FEE70907B4
:1024200000284FEA116104DB00F1E02080F800147D
:10243000704700F00F0000F1E02080F8141D704795
:102440006FF40041401804D0012803D0022801D0C5
:1024500008147047002070476FF40041401800D006
:10246000002070476FF40041401805D0012802D0C9
:10247000022801D0002070470120704770B5040089
:102480004FF0FF3511D020783A280ED10CA120460C
:10249000FEF76CF858B10CA12046FEF767F848B17A
:1024A0000BA12046FEF762F838B1284670BD48F20D
:1024B000010070BD48F2020070BD48F2030070BD1B
:1024C0003A535444494E00003A5354444F55540033
:1024D0003A535444455252006FF4004211140846D6
:1024E000704713466FF4004210B50C461114801863
:1024F00003D0012803D0022808D0084610BD2BB114
:1025000014F8010BFFF710FC5B1EF8E7002010BD6C
:102510008A68002A01DCFEF7CFB9521E8A604A6839
:10252000C0B2531C4B60107070470000FEF72EFFC6
:10253000FFF71CFFFFF70AFCFFF75AFCFFF796FDB9
:10254000FEF716FF00250446BFF34F8FBFF36F8FD2
:10255000234900200860BFF34F8FBFF36F8F214ADC
:10256000116841F400311160BFF34F8FBFF36F8FDB
:102570001C4970310860BFF34F8F081F43F6FF7E80
:102580000068174E1036C0F34E31C0F3C9030EEA8F
:102590004117184647EA807CC6F800C0401EF9D2B1
:1025A000491EF4D2BFF34F8F106840F480301060A2
:1025B000BFF34F8FBFF36F8F4FF47A76FEF7D8FEDD
:1025C000011BB14205D90446294607A0FDF70CFFBF
:1025D0000025FFF77FFEFFF735FD6D1CEEE70000DD
:1025E00050EF00E014ED00E04650533A2025640D12
:1025F0000A0000004FF04070E1EE100A70473A53B5
:102600005444494E003A5354444F5554003A53549D
:102610004445525200000000000000000001020387
:1026200004060708090000004826000800000020F2
:102630002C00000004020008742600082C00002072
:10264000EC0A000020020008010203040000000060
:10265000000000007C0000200100000010000000CD
:10266000000000000024F400000000000000000052
:042670000000000066
:04000005080001C925
:00000001FF
